:0400000088311C29FE
:1000080070082000A1007108A00080312100911E15
:1000180076282000911E762823009D1C24281D1276
:1000280019082000DE0023001D16013020004E07AD
:10003800F00000304F3DF1007008CE007108CF008D
:1000480023001D1D38289D139D17013020004E07E1
:10005800F00000304F3DF1007008CE007108CF006D
:10006800230019082000DE00230019082000DE0004
:100078005E080D3A0319492800306502031D462819
:1000880020306402031849285F280130EA00003054
:10009800EB0021009112CC3020006407860000306C
:1000A800653D870081016408E6006508E700E40112
:1000B800E501DE017528CC30640786000030653D17
:1000C80087005E0881006408E6006508E7000130E3
:1000D8006407F0000030653DF1007008E400710825
:1000E800E500911220002108F0002008F100090025
:1000F8000230FC004930FD00FD0B8028FC0B8028F5
:06010800000000000800E9
:0A010E002130FD00FD0B89280800D8
:0E0118003330FD00FD0B8E28000000000800B3
:1001260022006608F1000130F000710803199E28CC
:10013600F035FF3E99287008E800F009640884004D
:100146006508850070088005803084077008800582
:100156007C2068088004803084028C2068080005B2
:10016600E7006708003A013003190030E7007C20F9
:060176006708F00008001C
:10017C002000F801F9011030FC00710DF80DF90D9B
:10018C007408F8027508031C750FF9020318D528BA
:10019C007408F80775080318750FF9070310F00DAC
:0801AC00F10DFC0BC328080053
:1001B4002000F8010830FC00700DF80D7408F802F6
:1001C4000318E628F8070310F00DFC0BDE280800DE
:1001D40022006608F1000130F00071080319F528C7
:1001E400F035FF3EF0287008EA00F0097008E900D5
:1001F40064088400650885007008800580308407E1
:10020400E8016808073C031C1C296808F00067081B
:10021400F100700803191129F136FF3E0C29690811
:100224008005711C17296A0880048C206A088004E0
:0E023400E80A03298030840287208720080012
:1002420023009E1826290000212922006408230089
:040252009A00080006
:060256000000000008009A
:10025C002000FB01FA01F9018030F800F10CF00CE0
:10026C00031C41297408F90775080318750FFA0760
:10027C000318FB0A0310F01F49297408FA077508C4
:10028C000318750FFB07FB0CFA0CF90CF80C031C8C
:10029C0034297B08F3007A08F2007908F100780819
:0402AC00F000080056
:1002B00022005D08F2005E08F3007208F000730887
:1002C000F100F20A0319F30A70088400710885002E
:1002D000000803196C295D295D087202F0005E08B0
:0E02E000733BF1000130F0020030F13B0800EA
:1002EE0022005D0823009100920195131513151439
:0602FE001308F0000800E7
:100304002200E101053061020318922961085F07A8
:1003140086000030603D870030308100E10A842986
:1003240061085F0786000030603D87008101E103BA
:1003340000305E06031DA02900305D060319CE2996
:1003440061085F07E2000030603DE3000A30F4001A
:100354000030F5005D08F0005E08F100BE2078086A
:10036400F0007908F1003030F007220062088600BE
:100374006308870070088100E1030A30F40000304C
:10038400F5005D08F0005E08F100BE207008220050
:0A039400DD007108DE009A29080060
:10039E0022005D08393C031CDB2930305D02031C52
:0C03AE00DB290130F000DC29F001080020
:1003BA0020002230FC00F801F901FA01FB01FC03DC
:1003CA000319122A0310FB0CFA0CF90CF80CF30CA3
:1003DA00F20CF10CF00C031CE429FC030319042AA7
:1003EA007408F80775080318750FF90776080318D3
:1003FA00760FFA0777080318770FFB07E8297408BE
:10040A00F80775080318750FF90776080318760FA9
:0C041A00FA0777080318770FFB070800AB
:100426002200E001033060020318232A60085E07F9
:10043600860000305F3D870020308100E00A152AE3
:1004460060085E07860000305F3D87008101E0039B
:1004560060085E07E10000305F3DE2000A30F4000C
:100466005D08F000DA207808F0003030F00722004E
:100476006108860062088700700881000A30F4006F
:100486005D08F000DA2070082200DD007008003AEE
:0C049600031D4E2A502AE0032B2A080008
:1004A20022006108F000E10370080319862A5D0842
:1004B20084005E0885000008003A03196F2A5F086D
:1004C2008400600885000008F1005D0884005E0871
:1004D200850000087106031D6F2A7F2A5D088400CB
:1004E2005E0885000008F0005F088400600885004F
:1004F2000008F002F1010030F13B882ADD0A0319FD
:10050200DE0ADF0A0319E00A512AF001F1010800AC
:100512000C302200E4000030E500E6019320A63012
:10052200FD00FD0B922A00000C30E4000030E500D3
:10053200E6015530E700EA20DF01E0018030600685
:10054200F00080307002031DA82A08305F020318F1
:10055200D12A0C30E4000030E500E60101305D02F2
:10056200F00000305E3BF1000830F4000030F5008E
:100572002E212430F0070030F13D22005F08700781
:1005820084006008713D85000008E700EA20A6307B
:10059200FD00FD0BCA2A0000DF0A0319E00A9F2AA8
:0C05A200A630FD00FD0BD32A000008006D
:1005AE0022005D08F000F036F036F036F0363630C8
:1005BE0084008F308500700884070318850A0008B0
:1005CE00F0005E0886005F08870070088100013029
:1005DE005E07860000305F3D87000F305D05F0003E
:1005EE00363084008F308500700884070318850A22
:1005FE000008F0007008810002305E0786000030AF
:08060E005F3D87008101080037
:1006160022005D0884005E08850000085F06031D51
:10062600192B5D08F0005E08F1002B2B5D08F00029
:100636005E08F100DD0A0319DE0A700884007108FD
:1006460085000008F0007008031D0B2BF001F10176
:0206560008009A
:1006580022005F08F1000130F00071080319372B00
:10066800F035FF3E322B7008E3007009E200E1012B
:100678005D0884005E088500E0016008073C031CF3
:10068800662B6208800580308407620880052B216C
:10069800630880042B218030840263080005F00081
:1006A8000319622B6008F1000130F000710803198A
:1006B800602BF035FF3E5B2B7008E1048720872014
:0A06C800E00A412B6108F000080071
:1006D20022005F08F4006008F5005D08F2005E0881
:1006E200F3006108F0006208F1000130E10200301D
:1006F200E23B7008710403198F2B7408840075089B
:100702008500720886007308870000088100F20ADB
:100712000319F30AF40A0319F50A722B5D08F000B3
:060722005E08F100080072
:100728000D302200E40021210A302200E4002121BA
:020738000800B7
:10073A0022005D0823009100920122005E08230036
:10074A0093001513951315150B08F0008B135530EC
:10075A009600AA3096009514F01BB52B8B13B62B76
:0C076A008B171511951CBA2BB72B08003B
:1007760022005F088400600885000008F000700809
:100786000319D82B5F088400600885000008F00074
:100796005D0886005E08870070088100DD0A03197F
:1007A600DE0ADF0A0319E00ABB2B5D0886005E0835
:0607B6008700810108002C
:1007BC0022005D0884005E0885000008F0007008C7
:1007CC000319F42B5D0884005E0885000008E40022
:1007DC0021212200DD0A0319DE0ADE2B0630FD0082
:0807EC00FD0BF62B00000800D4
:1007F4002200E0015D0884005E0885000008DF0037
:100804005F08003A0319142C5F08E4002121220038
:10081400E00A60085D07840000305E3D8500000842
:06082400DF00022C0800B9
:10082A002200D901DA015408DB000030DB1BFF305B
:10083A00DC0080305406F0008030003A7002031861
:10084A00312CD90A0319DA0A5408003CDB00DC010E
:10085A000030D41BFF30DC3B5B08DD005508DE00AE
:10086A005608DF0013220430D7000030D800580899
:10087A00003C031D422C5708003C03185D2C570806
:10088A00550786005808563D870001305702F00088
:10089A000030583BF1007008550784007108563D36
:1008AA008500000881000130D7020030D83B3C2C7B
:1008BA0055088600560887002030810059085A04D6
:1008CA000319832CD701D801570855078400580803
:1008DA00563D85000008203A031D772CD70A0319D4
:1008EA00D80A692C0130D7020030D83B570855077F
:0E08FA0086005808563D87002D30810008000A
:100908002200D601D7015408F3005508F400540812
:10091800F5005508F600730884007408850000087F
:10092800203A031D9C2C56085704031D9C2CAD2C03
:100938000130D6000030D7007308840074088500A1
:10094800750886007608870000088100F50A0319F3
:10095800F60A7308F1007408F200F30A0319F40A9E
:1009680071088400720885000008003A031D8F2C66
:0A0978005408F0005508F1000800D3
:100982002200D001D101D201D301D51FD62C2100E2
:100992006C0886006D0887002D3081002200D40982
:1009A200D509D40A0319D50ADD2C21006C0886006A
:1009B2006D0887002030810022005408F00055089D
:1009C200F100F136F00CF136F00CF136F00CF136A4
:1009D200F00C7008D6005608D000D101D201D30124
:1009E2005408D7005508D8000F30D7050030D80575
:1009F2005708F0005808F1007130F4000230F50099
:100A02002E2170082200D7007108D8002030210062
:100A1200EC000130ED0022005608DD00013021001B
:100A22006C072200DE00003021006D3D2200DF0055
:100A3200132221006C082200DD0021006D08220033
:100A4200DE00FA232C30E400212122005708DD00C9
:100A52005808DE0021006C082200DF0021006D082A
:100A62002200E000822121006C082200DD0021002A
:100A72006D082200DE00582170082100EE00710886
:100A8200EF006E086C07F0006F086D3DF100023058
:100A9200700286000030713B8700810101306C07D3
:100AA2002200DD00003021006D3D2200DE00FA232D
:100AB2005008F0005108F1005208F2005308F30008
:100AC2001030F4002730F500F601F701DD21220095
:100AD2005708F4005808F500F601F701740870078A
:100AE200D0007508713DD1007608723DD2007708BA
:060AF200733DD300080073
:100AF800220054088400550885000008D600D70154
:100B08000030D70000305706031D8C2D20305606C4
:100B18000319972D00305706031D942D09305606EA
:100B28000319972D9B2DD40A0319D50A7C2DD801BA
:100B3800D901DA01DB0100305706031DA52D2D3040
:100B48005606031DAE2DDA0A0319DB0AD40A031967
:100B5800D50AB92D00305706031DB42D2B30560683
:100B6800031DB92DD40A0319D50A54088400550861
:100B780085000008D600D7010030D7005608DD00F0
:100B8800CF2170080319E22D5808F0005908F10028
:100B98000A30F4000030F5002E21303022005602D1
:100BA800F2000030573BF30072087007D800730852
:100BB800713DD900D40A0319D50AB92D5A085B0426
:100BC8000319EF2D5808003CF0005908031C013E9A
:100BD800F101F102F32D5808F0005908F10008005E
:100BE800D6302200DD008730DE00DE230C30E40042
:100BF8000030E500E60193200C30E4000030E50009
:100C0800E6013330E700EA200230FC00F130FD0055
:100C1800FD0B0C2EFC0B0C2E000000000C30DD0030
:100C28000030DE00DF012C2370082000DE002100E8
:100C38006C082200DD0021006D082200DE009130E2
:100C4800DF008E30E000BB23163021006C078600E1
:100C580000306D3D8700303022005407F0007008E6
:100C6800810020005E082200DD00A030DE00003098
:100C7800DF00D7225408F0005508F1001030F400C6
:100C88000030F5002E21A03070072200D600003079
:100C9800713DD7005608DD0020005E082200DE0006
:100CA8009D23013022005402F0000030553BF10032
:100CB8000830F4000030F5002E212430F007003011
:100CC800F13D70088600710887005E088100413098
:100CD800FC00EE30FD00FD0B6F2EFC0B6F2E0000AC
:100CE800113021006C072200DD00003021006D3D2D
:100CF8002200DE00A030DF000030E0000230E1001A
:100D08000030E200692301302000DF000030E000FD
:100D180000306002031D922E07305F020318F72E81
:100D28000C302200DD000030DE00DF012C237008CB
:100D38002000DE005F0822005607DD0020005E0864
:100D48002200DE009D23013022005402F000003012
:100D5800553BF1000830F4000030F5002E21243016
:100D6800F0070030F13D5F08700786006008713DAC
:100D780087005E0881004130FC00EE30FD00FD0B6D
:100D8800C32EFC0BC32E00005E082200DD00A0303D
:100D9800DE000030DF00D722173021006C07220068
:100DA800DD00003021006D3D2200DE0020005F08DC
:100DB800F0006008F1000230F4000030F5002E2148
:100DC80070082200DD077108DE3DA030DF0000302A
:100DD800E0000230E1000030E20069232000DF0A71
:100DE8000319E00A8C2E0C302200DD000030DE00F2
:100DF800DF012C2370082000DE005F082200560760
:100E0800DD0020005E082200DE009D230130220064
:100E18005402F0000030553BF1000830F400003077
:100E2800F5002E212430F0070030F13D073070071F
:100E380086000030713D87005E0881005E08220050
:100E4800DD00A030DE000030DF00D7222B3021008B
:100E58006C072200DD00003021006D3D2200DE001D
:100E6800A030DF000030E0000230E1000030E20096
:100E7800692321006C082200DD0021006D08220092
:100E8800DE00FA2394230830FB009D30FC00053077
:100E9800FD00FD0B4D2FFC0B4D2FFB0B4D2F0000C4
:0C0EA8000000220054082000E1040800B3
:100EB400003022005506031D612F0030540603192B
:100EC400992F540884005508850000080319992FA8
:100ED4005608DD005708DE0058217008E100540868
:100EE400DD005508DE005608DF005708E0005122F7
:100EF40000307106031D802F00307006031D872FFC
:100F04005408F0005508F1009B2F01305407DD0010
:100F14000030553DDE00560884005708850000085F
:100F2400DF000B237008D4007108D5005A2FF0019C
:040F3400F1010800BF
:100F380012001E00F003031D9C2FF103031D9C2FBC
:020F480008009F
:100F4A002000EA01EB01E601E70180306706F000C4
:100F5A0080307002031DB32F203066020318C72F9A
:100F6A00CC30660786000030673D8700810101307A
:100F7A006607F0000030673DF1007008E60071086E
:100F8A00E700AA2F230019082000DE00E401E5018A
:100F9A00E601E701DE01210091162000EE01EF01D2
:020FAA0008003D
:1010000022005408DD005508DE0080318922883135
:101010000C30E4000030E500E6014E30E70080319E
:10102000EA2088310230FC00F130FD00FD0B16286B
:10103000FC0B16280000000063280C30E400003090
:10104000E500E601200035082200E7008031EA20B3
:1010500088310230FC00F130FD00FD0B2D28FC0B27
:101060002D28000000000C30E4000030E500E6010F
:10107000200034082200E7008031EA2088317328FC
:101080000C30E4000030E500E601200023082200D7
:10109000E7008031EA2088310230FC00F130FD00A9
:1010A000FD0B5028FC0B5028000000000C30E40021
:1010B0000030E500E601200022082200E700803130
:1010C000EA208831732800305506031D6928013055
:1010D000540603191D2800305506031D71280230DF
:1010E0005406031940280230FC00F130FD00FD0BCE
:1010F0007728FC0B7728000000000C30E40000305B
:10110000E500E6017F30E7008031EA2088310230D7
:10111000FC00F130FD00FD0B8B28FC0B8B28000040
:1011200000005408DD005508DE0080318922883136
:101130000230FC00F130FD00FD0B9C28FC0B9C28CC
:10114000000000000C30E4000030E500E60148300B
:10115000E7008031EA208831EB30DD008E30DE00A0
:0E1160008031DE2388318031942388310800ED
:10116E0021302100C8000130C9006430CA000130AE
:10117E00CB00FF302000D200FF30D3000030D4006F
:10118E000030D500FF30D600FF30D7000030D80039
:10119E000030D900FF30DA00FF30DB000030DC0019
:1011AE000030DD0023009E1690309D0021008C142F
:1011BE000C142000911EE72823001908F000E028E7
:0211CE00080017
:1011D00022005408D500D6015508DD008031772162
:1011E000883170082200D700D80100305806031D4E
:1011F000FB2800305706031DFE281B298030F00015
:10120000803056067002031D07295508FF3C03185D
:101210000A291B295708E400803121218831220046
:10122000D50A0319D60A00305806031D19290030C3
:081230005706031DEC2808001D
:101238009E277030210099002F308C0023008C01EC
:10124800303024008C002200910192019D019D14F0
:101258009D171D152100EE01EF016E082000D0003A
:1012680021006F082000D1005008DF005108E0007D
:10127800E10120302100EC000130ED0023009F1532
:10128800CF309B009C011E15B7202000911E5029CD
:10129800230019082000DE00911E56292300190892
:1012A8002000DE000C302200E4008031212188314A
:1012B8000630FB001330FC00AD30FD00FD0B622949
:1012C800FC0B6229FB0B622900000000803194238B
:1012D800883125302200DD008F30DE008031DE23AA
:1012E8008831D401E8202030D400E8203030D40000
:1012F800E8205030D400E8207030D400E820803155
:101308009423883180319423883187302200DD008E
:101318008F30DE008031DE238831B030DD0080314F
:101328007721883170082000DE005E08283A03190A
:10133800A629FC302200DD008730DE008031DE2364
:101348008831E3292000DF01E00100306002031D3D
:10135800AF2908305F020318DE295F08B03E22007B
:10136800DD0080317721883170082000DE002430CC
:101378005F0786000030603D87005E0881005E08D8
:101388002200DD00A030DE000030DF008031D722EF
:101398008831A030DD000030DE008031FA2388314A
:1013A8002030E4008031212188312000DF0A031930
:1013B800E00AA92980319423883120006114C030C3
:1013C8002200DD0080317721883170082000DE009E
:1013D80080302200DD008F30DE008031DE2388314E
:1013E80020005E08283A0319022A93302200DD0003
:1013F8008F30DE008031DE2388313F2A2000DF0174
:10140800E00100306002031D0B2A08305F02031858
:101418003A2A5F08C03E2200DD00803177218831FA
:1014280070082000DE002C305F0786000030603D29
:1014380087005E0881005E082200DD00A030DE0023
:101448000030DF008031D7228831A030DD00003045
:10145800DE008031FA2388312030E40080312121F8
:1014680088312000DF0A0319E00A052A8031942315
:1014780088312000E11420302100EC000130ED001B
:101488008031A52788310B178B1723009F14200064
:10149800EC01ED01D001D10100306B06031D562A85
:1014A80001306A06031DCE2B00306D06031D5E2A2F
:1014B80000306C06031DCE2BCC302200D400003047
:1014C800D5004830D6000030D70080315A278831FF
:1014D80070082000EE007108EF006F08003C031D43
:1014E800772A6E08003C0318882A0130EC00003087
:1014F800ED006D302200DD008F30DE008031DE230C
:1015080088318031A5278831CC302200D4000030C2
:10151800D5004530D6000030D70080315A278831B1
:1015280070082000EE007108EF006F08003C031DF2
:101538009F2A6E08003C0318F32A02306E078400C5
:1015480000306F3D85000008DE0054302200DD00C9
:101558008F30DE008031DE238831D030D400003077
:10156800D50080317C25883170082000E2007108A0
:10157800E3007F30F000803063067002031DC62A46
:101588006208C93C0318F02A80306306F0008030F6
:101598007002031DD12A7D3062020318F02AE72A5F
:1015A8006208B50001302200D4000030D5000020C8
:1015B800F02A20006208A30002302200D400003084
:1015C800D5000020F02A20005E08313A0319D42AF9
:1015D8005E08323A0319DD2A8031A5278831CC30DC
:1015E8002200D4000030D5003A30D6000030D700B1
:1015F80080315A27883170082000EE007108EF000A
:101608006F08003C031D0A2B6E08003C03185E2B74
:1016180002306E07840000306F3D85000008DE0050
:1016280061302200DD008F30DE008031DE2388311A
:10163800D030D4000030D50080317C258831700846
:101648002000E2007108E3007F30F000803063067C
:101658007002031D312B6208C93C03185B2B8030D4
:101668006306F00080307002031D3C2B7D3062025F
:1016780003185B2B522B6208B40001302200D400FF
:101688000030D50000205B2B20006208A200023049
:101698002200D4000030D50000205B2B20005E081B
:1016A800313A03193F2B5E08323A0319482B80312F
:1016B800A5278831CC302200D4000030D500363040
:1016C800D6000030D70080315A27883170082000B2
:1016D800EE007108EF006F08003C031D752B6E08C3
:1016E800003C0318CE2B04306E07F00000306F3D2D
:1016F800F10070088600710887003F30810070088B
:1017080084007108850000080319CE2B03306E078A
:10171800840000306F3D85000008DE00463022005E
:10172800DD008F30DE008031DE23883120005E0846
:101738002200E400803121218831803194238831CE
:10174800303020005E02E200E3010030E33B8030ED
:10175800F000803063067002031DB42B6208003C61
:101768000318CB2B80306306F00080307002031D15
:10177800BF2B033062020318CB2B62082200D4006F
:10178800200063082200D5008031F425883180319B
:10179800A527883100306B06031DD42B01306A065B
:1017A8000319DF2B6508003C031DDC2B6408003C93
:1017B800031CDF2B372C00306D06031DE52B013091
:1017C8006C06031D372C0630FB001330FC00AD30CF
:1017D800FD00FD0BED2BFC0BED2BFB0BED2B0000A7
:1017E8000000CC302200DD000030DE008031FA231A
:1017F8008831803194238831CC302200D4000030E5
:10180800D5003D30D6000030D70080315A278831C6
:1018180070082000EE007108EF006F08003C031DFF
:10182800172C6E08003C0318372C0230FB000430DC
:10183800FC00BA30FD00FD0B1F2CFC0B1F2CFB0B12
:101848001F2C000078302200DD008F30DE00803150
:10185800DE2388318031942388312000EC01ED01AA
:101868008031A527883100306D06031D3D2C0130DD
:101878006C06031D482C8031A527883123009F144E
:1018880000000000630000008031A52788319B30EC
:101898002200DD008F30DE008031DE238831200019
:1018A80050082200DD00A030DE000030DF0080316B
:1018B80013228831A030D4000030D5008031842430
:1018C8008831A030DD000030DE00803158218831B9
:1018D8007008033C2100EE007108031C013EEF0173
:1018E800EF026F08003C031D7B2C6E08003C0318B8
:1018F800892C20302200E4008031212188310130F8
:101908002100EE020030EF3B752CA0302200DD00F4
:101918000030DE008031FA2388312000611C892DD7
:1019280001302200DD000030DE008031892288315C
:101938000C30E4000030E500E6014430E700803177
:10194800EA2088311A30FC00F830FD00FD0BAA2C83
:10195800FC0BAA2C00000130DD000030DE008031D5
:10196800892288311A30FC00F830FD00FD0BBA2CB2
:10197800FC0BBA2C00000C30E4000030E500E60156
:10198800BE30E7008031EA2088310C30DD000030BD
:10199800DE00DF0180312C23883170082000E80048
:1019A800E9010C302200DD000030DE00DF0180316B
:1019B8002C2388317008F200F10171082000E80733
:1019C8007208E93D0C302200DD000030DE00DF0146
:1019D80080312C23883170082000B5000C3022009B
:1019E800DD000030DE00DF0180312C2388317008F3
:1019F8002000B4008E302200DD008F30DE00803100
:101A0800DE2388311A30FC00F830FD00FD0B0A2D6A
:101A1800FC0B0A2D0000200068082200D4002000DA
:101A280069082200D5008031C12488312030210086
:101A3800EC000130ED00A0012200A00121006C089B
:101A48002200DD0021006D082200DE000230DF00E8
:101A58008F30E0008031BB23883120003508220018
:101A6800D400A030D5000030D6008031152488314C
:101A7800043021006C072200DD00003021006D3D9C
:101A88002200DE00A030DF000030E0000430E1007A
:101A98000030E200803169238831200034082200B8
:101AA800D400A030D5000030D6008031152488310C
:101AB8000C3021006C072200DD00003021006D3D54
:101AC8002200DE00A030DF000030E0000430E1003A
:101AD8000030E20080316923883121006C0822003F
:101AE800DD0021006D082200DE008031FA238831F4
:101AF8000930FB001E30FC00E430FD00FD0B822D98
:101B0800FC0B822DFB0B822D00002000E11C742EA3
:101B180002302200DD000030DE0080318922883169
:101B28000C30E4000030E500E6014430E700803185
:101B3800EA2088311A30FC00F830FD00FD0BA22D98
:101B4800FC0BA22D00000230DD000030DE008031E9
:101B5800892288311A30FC00F830FD00FD0BB22DC7
:101B6800FC0BB22D00000C30E4000030E500E6016B
:101B7800BE30E7008031EA2088310C30DD000030CB
:101B8800DE00DF0180312C23883170082000E80056
:101B9800E9010C302200DD000030DE00DF01803179
:101BA8002C2388317008F200F10171082000E80741
:101BB8007208E93D0C302200DD000030DE00DF0154
:101BC80080312C23883170082000A3000C302200BB
:101BD800DD000030DE00DF0180312C238831700801
:101BE8002000A20097302200DD008F30DE00803117
:101BF800DE2388311A30FC00F830FD00FD0B022E80
:101C0800FC0B022E0000200068082200D4002000EF
:101C180069082200D5008031C12488312030210094
:101C2800EC000130ED00A0012200A00121006C08A9
:101C38002200DD0021006D082200DE001430DF00E4
:101C48008F30E0008031BB23883120002308220038
:101C5800D400A030D5000030D6008031152488315A
:101C6800043021006C072200DD00003021006D3DAA
:101C78002200DE00A030DF000030E0000430E10088
:101C88000030E200803169238831200022082200D8
:101C9800D400A030D5000030D6008031152488311A
:101CA8000C3021006C072200DD00003021006D3D62
:101CB8002200DE00A030DF000030E0000430E10048
:101CC8000030E20080316923883121006C0822004D
:101CD800DD0021006D082200DE008031FA23883102
:101CE8008031942388312000D00A0319D10AFF30AB
:101CF800D0050030D1051530FB004B30FC00BE305C
:101D0800FD00FD0B852EFC0B852EFB0B852E0000A0
:041D1800502A8D2E92
:101F3C00BF3084008E3085002C30F0000130F10071
:101F4C00223086000030870080319C2788310800C1
:100FAC000D340A34313420347334653475346C3474
:100FBC0020344434533431343834423432343034C1
:100FCC00203464346F3469347434203465347434AC
:100FDC0072346534203463346F346E346E3465345B
:0C0FEC0063347434E9340D340A340034EA
:080FF8003F340D340A340034CB
:101D220044346134743461343A3420344634613496
:101D32006D3469346C34793443346F3464346534CB
:101D420020342E342E342034493444342E343D345D
:101D52002034783478347834783478347834783479
:101D620078347834783478347834203443345234C4
:0C1D720043343D3420342E342E34003431
:021D7E000E3421
:021D8000143419
:101D820000340034003400340034003400340034B1
:101D920000340034003400340034003400340034A1
:021DA2000F34FC
:021DA4001334F6
:081DA6004934443423340034B5
:061DAE0054344C340034F3
:101DB4002E34573441344B34453455345034003484
:061DC400543448340034E1
:0C1DCA0053344C3445344534503400345C
:101DD60020342D343E34733474346F3472346534A5
:101DE6006434203469346E3420344434533431340A
:0E1DF60038344234323430340D340A34003480
:101E04003B34483431343D342E342E342E342E3485
:101E14003B344C3431343D342E342E342E342E3471
:041E24003B34003417
:101E28003B34483432343D342E342E342E342E3460
:101E38003B344C3432343D342E342E342E342E344C
:021E4800003464
:101E4A00563465347234733469346F346E342034E2
:101E5A003134373430343334303433340D340A3493
:021E6A00003442
:101E6C00303431343234333434343534363437342A
:101E7C0038343934413442344334443445344634B0
:101E8C005234653463346834653472346334683482
:0C1E9C00653420344934443423340034CD
:101EA80053346534753469346C34203448346134BF
:0A1EB800753474340D340A3400341C
:101EC20053346534753469346C34203442346134AB
:081ED20073340D340A340034AE
:101EDA0053344C3445344534503449344E34473401
:061EEA000D340A3400343F
:101EF00057344F3452344B3449344E344734003421
:0E1F0000493444342034233432342034003445
:0E1F0E00493444342034233431342034003438
:0A1F1C003B34543431343D340034BA
:081F26003F340D340A3400348D
:081F2E00543432343D34003418
:061F36006A343D34003462
:020000040001F9
:04000E00E429FF38AA
:020000040001F9
:10E0000043006F006D00700069006C0061007400D7
:10E0100065007500720020004D0069006B00720001
:10E020006F0043002000200037002E0030002E003B
:10E03000310020000D000A00000020002000200018
:10E0400041006C0069006D00200033002C0033009B
:10E05000560020000D000A000000200020002000D3
:10E0600050004900430031003200460031003800C2
:10E0700034003000200065007400200032002000D1
:10E0800053006F006E0064006500200044005300E0
:10E09000310038004200320030000D000A0000005C
:10E0A00041006C00610072006D00200054004800C7
:10E0B0003100200065007400200054004C00310045
:10E0C0002000540048003200200065007400200049
:10E0D00054004C00320020000D000A000000200017
:10E0E00043006400650073002000440049005300B1
:10E0F00050004F0020003A00200020000D000A00D0
:10E100005400480031003D00200020006F007500E1
:10E11000200054004C0031003D0020000D000A009A
:10E1200053004C0045004500500020002000200016
:10E130002000200020002000200020000D000A0008
:10E140002E00570041004B004500550050002000B4
:10E15000200020002000200020000D000A00000008
:10E1600020002000200020002000200020002400AB
:10E17000200020002000200020002000200020009F
:10E180002000200020002000200020002000B800F7
:10E19000200020002000200020002000200020007F
:10E1A000200020002000200020002000200020006F
:10E1B000200020002000200020002000200020005F
:10E1C000200020002000200020002000200020004F
:10E1D000200020002000200020002000200020003F
:10E1E0007000610075006C0066006A0075006A00CE
:10E1F0006F00400066007200650065002E000000A0
:00000001FF
